:030000000219FDE5
:03000B000200AA46
:03002B0002018A45
:03005B0002033C61
:030073000203295C
:1000800002030406080C10182030406080040608A3
:100090000C10182030406080A0C00003070F1F0D17
:1000A0000D0403060D0503030202C2AF306308C24C
:1000B0006385798AD2AF32C0D0C0E0206221E525C5
:1000C0006016E473E525F4C3334009758A00D263F2
:1000D000F57901D6F58AD262D0E0D0D0D2AF32C362
:1000E000E526334009758A00D263F57901F0F58A77
:1000F000C262E526F4603030682620720DD0E0D070
:10010000D0C295C294C293D2AF32C295C294C29368
:10011000206F0D20650A7414D5E0FDE57BF4529044
:10012000D0E0D0D0D2AF32758A00D263757900C2E8
:100130008DD262212001C4306805206502D295016C
:10014000C4306805206502D29401C430680520657A
:1001500002D29301C4D29230680A2065077410D588
:10016000E0FDD29501C4D29130680A206507741071
:10017000D5E0FDD29401C4D290D29230680A2065B5
:10018000077410D5E0FDD29301C4C2AFC2AD53E6EF
:10019000EFC0D0C0E0D2D3D2AFE57A6009E5776096
:1001A00005757700412C757701C2CEE52A600720DE
:1001B000744F152A41017800790020742EE58030B3
:1001C0007E01F430E70278FF53DACF207E0343DA72
:1001D00020307E0343DA10C2D8C271E580307E0140
:1001E000F430E70279FFC3E89970CB306103752AD8
:1001F00040207403752A40885CD270E86003755F04
:100200000020740DE52B6004152B411143DA01C267
:10021000D82070024124A85C206102C270207402C0
:10022000412288227882B6040385222420CF0AD076
:10023000E0D0D043E610D2AD32C2CF053AE57A60C5
:1002400009E5786005757800611F7578017802E529
:100250002A6005307402152AC3E55C9401400575D7
:100260005F004175756000756900E55F2401F55F09
:100270005003755FFF7982B7020D306E1DC3E52212
:1002800094324016854C227982B7030E306E0BC330
:10029000E52294324004798E8722C3E523952260BB
:1002A000084004152341A90523D8CA0569E56970EA
:1002B000021569D56A69756A017808E56B60497845
:1002C00005C3E569956B4057C3E569956C5008789F
:1002D00001756A030202E3C3E569956D5005780173
:1002E000756A01C3E5629524401E7982B7040261F4
:1002F00014206E14852462E569046003856B6975BA
:100300006A0175233C02031FE5622850057562FFF0
:100310006114F562E5620470067560FF7569FFD0CF
:10032000E0D0D043E610D2AD32C2AF53E67F759233
:10033000FA7593FFC260759104D2AF32C2AF53E633
:10034000EFC2ADC0D0C0E0C0F0D2D3D2AFA8FBA9FD
:10035000FCE57A6007C3E913F9E813F8C2D83071F5
:100360000261AE53DACF207E0343DA10307E0343BE
:10037000DA20D271E580307E01F420E702618588C1
:10038000278928A19353DACF207E0343DA20307ED9
:100390000343DA10C2D8C271307402A17F7800E53D
:1003A00080307E01F430E702A17F885CA16753DAD8
:1003B000CF207E0343DA20307E0343DA10C271205F
:1003C0006102818753DACF207E0343DA10307E0347
:1003D00043DA20C2D8D27188578958C3E89555F8B6
:1003E000E99556F97B007E087A00C3E8948CE9947D
:1003F000005005755B008179882178A2E6A821600C
:1004000055C3E894C8E994005008E4D2E4FB7A0AA2
:100410008154C3E89468E994015008E4D2E3FB7A7C
:100420000F8154C3E894D0E994025008E4D2E2FB6F
:100430007A1E8154C3E894A0E994055008E4D2E1FF
:10044000FB7A3C8154C3E89498E994085008E4D2BC
:10045000E0FB7A787E00C3E89559FCE9955AFD30B7
:10046000E70AECF42401FCEDF43400FD755B00C3F5
:0D047000EC9AED9E5003755B018859895A86
:10047D008557558558567802A167C3E89527F8E941
:10048D009528F9307C02A14B307B02A14B307A02CA
:10049D00A14420750281AAE9FDE8FC81C9E9C313D5
:1004AD00F9E813F8307902A144E9C313F9E813F818
:1004BD00307802A144E9C313FDE813FC20612CC37D
:1004CD00EC941CED9402400281E0ED701EC3EC949F
:1004DD00C850180529E52970021529C3E529940A84
:1004ED005002A17F755C00D270A17FE529600215D5
:1004FD00297400207F037896E624FAFEE43400FF89
:10050D00C3EC9EFCED9FFD500678007900A14BC316
:10051D00EC94FFED9400400678FF7900A14BEC853B
:10052D0072F0A4C5F0A2F733F87900400302056715
:10053D0078FF7900020567E9C313F9E813F8307CF9
:10054D000EE9600278FFC3E81338F8E43400F9C30C
:10055D00E894FFE99400400278FF885CD270206136
:10056D0002A17F741FF4552F4BF52FC274EB70024F
:10057D00D274752A40307403752A0A306102A19332
:10058D0020740353DAFE207403752B20D0F0D0E0D5
:10059D00D0D0D2AD43E6103279010205C379030202
:1005AD0005C3790A0205C3791E0205C379640205E4
:1005BD00C379C80205C37817E4D5E0FDD8FAD9F69A
:1005CD00227A147B780205EA7A107B8C0205EA7A8E
:1005DD000D7BB40205EA7A0B7BC80205EAE573D5FB
:1005ED00E001227902E4D291D5E0FDD294D5E0FD6F
:1005FD00C294D5E0FDC291D5E0FDE920E002D2958F
:10060D0030E002D293E573D5E0FDE920E002C2951A
:10061D0030E002C2937496D5E0FDD9C9EAF8D5E071
:10062D00FDD8FBDBB8D29122C37C007D0075F000B4
:10063D0005F0EA33FAEB33FB50F6EB13FBEA13FA52
:10064D00C3E9FFE8FEE89AF8E99BF95004EFF9EEEB
:10065D00F8B3EC33FCED33FDD5F0DFEDF9ECF8221A
:10066D00E889F08A20D2D4F8A9F07B0030F70B7B13
:10067D00FFF42401F8E9F43400F9E88520F0A4AD85
:10068D00F0F8E98520F0A4AFF0FEED2EF974003FEF
:10069D00FA7C04C3EA13FAE913F9E813F8DCF48BD6
:1006AD00F030F70AE8F42401F8E9F43400F9E889A8
:1006BD00F0C2D4F8A9F0227882B60403020763C30E
:1006CD00E55C9419401EE52D54067018206E3678A1
:1006DD00057994E7146007780A1460027812C3E56F
:1006ED004198401F306E098564627569FF756A0116
:1006FD00852224E4F544F545F546F547F548C26EE7
:10070D00020763D26E7994E7147013E523F4333343
:10071D00F913F8E9540104F9E854FE020757E714F8
:10072D00147014E523F4333333F913F8E954030447
:10073D00F9E854FC02075FE523F433333333F9133F
:10074D00F8E954070404F9E854F8C39440F8E9941F
:10075D0000F98844894522C3E54113F9E54013F8B2
:10076D00C3E54498F8E54599F9500CC3E89480E940
:10077D0094FF401602079BC3E8947FE99400500351
:10078D0002079B787F790002079B788079FF884963
:10079D00894A22E5492546F8E54A3547F9854A2033
:1007AD00E4300701F43548FA30E709C3EA94F04024
:1007BD00150207D9C3EA940F50030207D978FF79C0
:1007CD00FF7A0F0207D9780079007AF0C3E52495F6
:1007DD0061500AC374019524500B0207F7E54A20B6
:1007ED00E70E0207F7E54A30E706884689478A484B
:1007FD002278A5E6FAC3E54933F8E54A33F912063E
:10080D006DE930E70BC3E89480E994FF40130132A2
:10081D00C3E8947FE9940050020132787F7900019A
:10082D0032788079FFE820E715C3E52398F8400971
:10083D00C3E8940140030208597801020859E8F40D
:10084D0024012523F8400302085978FF884B2278AC
:10085D00A6E6FAA847A94812066DE930E70CC3E8E9
:0F086D009401E994FF401602088EC3E894FFE956
:10087C009400500302088E78FF790002088E7801EC
:10088C0079FFE920E715C3E54B98F84009C3E894D4
:10089C000140030208B578010208B5E8F4240125EB
:1008AC004BF840030208B578FF88242278FF2069B2
:1008BC002879A1E76023E541601F74FF8541F0842E
:1008CC008539F0306A0375F005A4F8C5F06002783C
:1008DC00FFC3E895645002A864886322C3E5409482
:1008EC00C8E5419400E56350031401F9046002F576
:1008FC0063227883E6F520120F9975E8901205A50E
:10090C0075E89030EDFDA8BDA9BE121044756E00BF
:10091C00756F00C3740013FD7400606613FC7400E3
:10092C002CFC74003DFDECFAEDFBC3E89AE99B400E
:10093C0014E56E2400F56EE56F3400F56FEA2CFAC1
:10094C00EB3DFB80E5AE6EAF6FC3E56F13F9E56E63
:10095C0013F8C3E913F9E813F87A03C3E913F9E8B8
:10096C0013F8DAF7AA201A7009756E00756F000279
:10097C00098E1AEA6008EE28FEEF39FFDAF88E6E5F
:10098C008F6F2275E890227883E6FF30EDF9A8BDD1
:10099C00A9BE0570C3E57094084052757000E9FA61
:1009AC0079A0E76044EA7007E571601B0209C7C3D0
:1009BC00E895716010E5715006600C140209D304BF
:1009CC0060F90209D3E571F571C39472401B75612E
:1009DC00C0C394044013756180C39404400B7561CB
:1009EC0040C39404400375610075BB0622EFC394A9
:1009FC0001601F7400601BC3E894FFE9940350125C
:100A0C00C3E8956EE9956F5009E561600C156102BC
:100A1C000A25E561F460020561A861C3E5249850DC
:100A2C0002A824C3E89562400AA862E562F4600358
:100A3C0085626188258826E570B4070375BB102292
:100A4C00743279A787F0A4C5F0A2F733F8C3E89500
:100A5C00614002A86188228824882588268864221F
:100A6C007540007541F022C2AF75C820A8CCA9CD45
:100A7C00AA3A30CF010A75C824D2AFC3EA13FAE9F7
:100A8C0013F9E813F8AB3BAC3C883B893CC3E89BBF
:100A9C00F8E99C20690A547FF9306602619241ECB6
:100AAC00AD3D8A3DF9EA9D547FFA600678FF79FFE7
:100ABC0041D1AE3EAF3F8B3E8C3FA83BA93CC3E837
:100ACC009EF8E99FF9C3E54113FBE54013FAE82AC8
:100ADC00F540E93BF54150067540FF7541FF613922
:100AEC00AA40AB41AC40AD417E047F02C3EB940401
:100AFC00400D1E1FC3EB94084005206A021E1FC345
:100B0C00ED13FDEC13FCDEF7C3EA9CFAEB9DFBEF57
:100B1C006009C3E913F9E813F8DFF7EA28FAEB39AF
:100B2C00FB8A408B4150067BFF8B408B41C3EB947F
:100B3C00025002D2663069047F0361647892E6FF4A
:100B4C00C3E537948240110FC3E53794A040010FE1
:100B5C00C3EF940640027F057E02E541C4540FF9B1
:100B6C00E541C454F0F8E540C4540F28F8C3E89E9E
:100B7C00FAE99400FB4009C3EA9402EB9400500498
:100B8C007A02E4FB61DEAA40AB41EBC4FEEAC4543A
:100B9C000F4EFCC3EA9CFAEB9400FBC3E813C3139F
:100BAC00F8EA28FAEB3400FB8A408B41C3EB940241
:100BBC004002C2667802EBC4FE7B00EAC4540F4EBE
:100BCC00FAC3EA98FA4005C3940250027A0278926A
:100BDC00E6FF30600261DE855192855293D260430C
:100BEC00E680C3E49AF8E49BF9C3E833F8E933F9F7
:100BFC003066028171E8FAE9FBD3E913FDE813FCD6
:100C0C0088518952C3EF94036038EF20E00DE82C33
:100C1C00F8E93DF9ECFAEDFB020C3AE828F8E93971
:100C2C00F9C3E82402F8E93400F97AFE7BFFC3EF3C
:100C3C009403400E8A538B54884D894E8C4F8D50A3
:100C4C0081A5885389548A4D8B4E8C4F8D503069B9
:100C5C00127553F07554FF754FF07550FF7551F0C8
:0F0C6C007552FF81A5E8FAD3E813FC8851C3EF56
:100C7B0094036020EF20E007E82CF8ECFA8191E870
:100C8B00282402F87AFEC3EF940340088A53884D58
:100C9B008C4F81A588538A4D8C4FE568C333500226
:100CAB00646BF56830600281AF753402D26043E645
:100CBB0080E52D5406602DA840A941C3E913F9E83E
:100CCB0013F8306904E92440F9C2AF53E67F7591FC
:100CDB0000C3E498F594E499F595759104D26043BB
:100CEB00E680D2AF22D264754300752000306C03CE
:100CFB00752040020D0FD264754300752040306C97
:100D0B000375200078017901206620E52D540660DB
:100D1B0002C2647914E541C313700104F8C394143F
:100D2B0040027814306904781B791BC3E833F8C38D
:100D3B00E933F9206010E543600C306903D53404C6
:100D4B00D26DA1C591B70543E59B5440B52002A1D7
:100D5B00AF30690908C3E899400118A13E20640A25
:100D6B0008C3E8994002A10FA13EC264C2AF53E68B
:100D7B007F7591003066127594007595F07591042E
:100D8B00D26043E680D2AFA10FE5417EFFC3334073
:100D9B0009C3334005C3334001FEC3E49E75940081
:100DAB00F595A188C3E53394015002A10F3064027D
:100DBB00A10FD802A1C3A13EC26DC2AF53E67F758E
:100DCB009100855394855495759104854D92854E6C
:100DDB0093D26043E680D2AFE52D54066008206ABB
:100DEB00020533020E01306D0D206C0A20640715CD
:100DFB008115810216BD2278003064027801E53737
:100E0B0075F007A4F9E5F028F5F0E9A2F013A2F1CB
:100E1B0013A2F213F537C394785003753778C3E5F3
:100E2B003795384008D265C295C294C293306002A0
:100E3B00C138854F92855093D26043E68022207D46
:100E4B0016C2AF754202D291C292306202D293D2D5
:100E5B00AF759F11021041C2AF754202D291C29081
:100E6B00306202D295D2AF759F110210413072459C
:100E7B00207D22C2AF754203900166757B02C2933F
:100E8B00D290D292306204D294C198C291D2AF75F3
:100E9B009F01021041C2AF754203900166757B0240
:100EAB00C295D292306204D294C1B8C291D2AF75BE
:100EBB009F21021041207D17C2AF75420390014163
:100ECB00C293306202D294D2AF759F01021041C21D
:100EDB00AF754203900141C295306202D294D2AFFA
:100EEB00759F21021041207D16C2AF754204D2922C
:100EFB00C290306202D294D2AF759F21021041C2D0
:100F0B00AF754204D290D292C292306202D294D286
:100F1B00AF759F01021041307243207D20C2AF7527
:100F2B004205900155757B04C294D291306204D274
:100F3B0095E140C292D2AF759F11021041C2AF75BD
:100F4B004205900177757B01C294D291306204D235
:100F5B0093E160C290D2AF759F11021041207D17B3
:100F6B00C2AF754205900137C294306202D295D25E
:100F7B00AF759F11021041C2AF75420590014BC274
:100F8B00943062EBD293D2AF759F11021041207D4A
:100F9B0018C2AF754206D290D292C291306202D281
:100FAB0095D2AF759F01021041C2AF754206D29226
:100FBB00C291306202D293D2AF759F2102104130A1
:100FCB007246207D20C2AF754201900177757B017F
:100FDB00C295D292306204D293E1E8C290D2AF753F
:100FEB009F21021041C2AF754201900155757B04E0
:100FFB00C293D290D292306205D29502100BC2925C
:10100B00D2AF759F01021041207D17C2AF7542010F
:10101B0090014BC295306202D293D2AF759F2102E1
:10102B001041C2AF754201900137C293306202D2B8
:10103B0095D2AF759F01C26522900135757B00C2B9
:10104B0095C294C293D292D291D290C262227880EE
:10105B0076070876070876010876040876FF087687
:0F106B00FF08760A087602087601087601788C6D
:10107A0076010876000876B40876FF0876FF0876C7
:10108A00FF0876030876FF0876010876FF087625BA
:10109A000876D00876780876C80876040876FF08B5
:1010AA00760108760008767A08760A0876010876C4
:1010BA00010876000876FF087600227887E6FFC2E4
:1010CA0072BF0302D2727888C27DE630E102D27D15
:1010DA00C27E7889E630E102D27EC3EF94026008CC
:1010EA00758E01D2730210F7758E00C27322788052
:1010FA00E6149000809378A5F67881E61490008033
:10110A009378A6F67886E61490008D9378A7F678F9
:10111A009FE6F87005756B00213EC3E89411400202
:10112A007811E82828F56B256B256B28F56C256B5B
:10113A002828F56D7886E6F539C394025003753987
:10114A0002789CE67538FFB402037538A0B403032D
:10115A0075388278A3E61490009A93F566114422B2
:10116A00227896E6FA7897E6FB7888E6B40305C310
:10117A00EB940EFB307F047A007BFFC3EB9AFCC32F
:10118A00948250027C827572000572EC8572F0A41A
:10119A00C3E5F0947D40F222D27F316B1205B4127E
:1011AA0005B47A007B007C101205AAE55C2AFA7461
:1011BA00003BFBDCF37C04C3EB13FBEA13FADCF71A
:1011CA00FEC27F316B22757C00757D00E5EF20E65B
:1011DA00037520000520903FFFE520146006901F4C
:1011EA00FF1460009304600375EF1653D9BF75812D
:1011FA00C043FF801205A575EF0643B203E5B32489
:10120A000220E70DF521E5E320E0068521B343E35B
:10121A000111447580FF75A40075F19075D47F752E
:10122A00908775A5BF75F2BF75D50075A60175E2E1
:10123A00411144E4F8F6D8FD756801115912171BDB
:10124A0078988673753001C2AF1205BE1205CE12A8
:10125A0005B41205D51205B41205DC1205B412182C
:10126A004E1205BE1205BE1205B9C2AF757C0075D5
:10127A007D0078FA79FA308707D9FBD8F7021C0083
:10128A0011C511F8316A316B78988673114475A9C2
:10129A000075B680757A0075881075890275C8243C
:1012AA0075910475D84075A82275B80275E69075CF
:1012BA009B80759D0075D10E75BC5875BB0675BAB5
:1012CA001175E8801205A5D2AF1208FE75360053D3
:1012DA00DACF207E0343DA20307E0343DA1043DA82
:1012EA0001C2D8C2711205BED2617B037A0CE55BDA
:1012FA0070077A0CDB030212741205B42070030221
:10130A001274C270E55CC3940240E1E52F541F8554
:10131A005E5DF55EB55DD5DAD5C26153DACF207E62
:10132A000343DA20307E0343DA10C2D8C27178A2AE
:10133A00E67008D274E52F54E0F52FC275752900BE
:10134A001205B9307409C3E529940A4002D275120C
:10135A0005AA78023074027800C3E55C9840F0C2AE
:10136A00AF1205CE1205CE1205CED2AF1205BE754A
:10137A004C001205AA788CE6C39401500302146942
:10138A00E530C394015003021469757CA5757DF19B
:10139A00207435C3E55C94FF5003021469C2AF128E
:1013AA0005E3D2AF1205B9C3E55C940150EFC2AFB1
:1013BA001205CE1205AF1205CED2AF1205B9C3E59A
:1013CA005C94FF40E90218D37F05D27F316B120586
:1013DA00B9C2AFC27F316BAE5CC3E55C947FD2AF5A
:1013EA00500281791205A5C2AF1205E3D2AFDFDA46
:1013FA0031A2C3EE94057897F61205BE1218567FED
:10140A000AD27F316B1205B9C2AFC27F316BAE5CB3
:10141A00C3E55C947FD2AF50E61205A5C2AF1205B0
:10142A00CE1205AF1205CED2AFDFD631A2EE24031B
:10143A007896F6F87997E7C394824003985006E8BD
:10144A0024827897F61205BE1217681218851205BB
:10145A00B9316BC3E55C94FF500261940218D375ED
:0F146A007C00757D00C3E55C954C4003855C4CB0
:101479001205B978017988E7B403027805C3E55CF8
:10148900984002617CC2AF1205E31205E31205E33D
:10149900D2AF1205BE753000E4F531F5320531E5FC
:1014A90031F4703E0532789AE67819146012783270
:1014B90014600D787D14600878FA146003753200A1
:1014C900C3E53298401C11441205A5153275310047
:1014D90078998673C2AF1205E3D2AF7898867312F2
:1014E90005B91205AFE52A70053074024174780117
:1014F9002074027806C3E55C9840A21205B9E52A72
:101509007003021274C2AF1144E4F522F523F524E5
:10151900F525F526F567D2AF7885E6C333F565E499
:10152900F544F545F546F547F548F570F52CF52DE3
:10153900F53775700875BB101205A512098F30EDC6
:10154900FDA8BDA9BEE97001F888711209937570EB
:101559000875BB1011C5C2AF7561FF120A4C85220F
:1015690061852262852263D2AF75220175240175D6
:101579002501752601856069756A0175B69075A999
:1015890003757A017888E6B40307C27D307602D202
:101599007DD268D269753300120F99120FCA120AE7
:1015A9006C120A73120A6C120A73120A6C120D0178
:1015B9001206C4120E02120E49120A73120CF030EE
:1015C9006E031207642066031208B8306603120816
:1015D900E8120E02120E78120A73120D01306E0310
:1015E9001207A0120E02120EF1120A73120CF03039
:1015F9006E031207FE120E02120F22120A73120D47
:1016090001306E0312085C120E02120F99120A734E
:1016190012098F120CF0120E02120FCA120993123C
:101629000A7330692C856461856462856069756AAD
:101639000179187A0CC3E533994009C269D26A8ADB
:101649003502165AC3E55C940140030215B6021629
:10165900C5306A25206C22E535147006C26AD26B42
:10166900A1B6F535C3E55C940140030215B6788847
:10167900E6C3940360030216C5753600C3E55F949B
:10168900014009856462856069756A0178FA79A4FF
:10169900E760027803C3E55F985021307404E52AB6
:1016A900601A78F0306C058564617820C3E541984B
:1016B9005002A1B60536E55C6002C1C8753600C2A4
:1016C900AF11447887E6FE760211C57887EEF6E415
:1016D900F522F523F524F525F526F565752C007514
:1016E9002D0075A90075B680757A00D2AF1205B9BB
:1016F900114478A4E66006C292C291C29030740681
:10170900E52A70024174788DE6C39401400261595B
:1017190081A1901A0D78201217AAE520B4A50CA36F
:101729001217AAE520B45A03021748757CA5757DDE
:10173900F11159121768757C00757D0002176790C1
:101749001A0378807B0A1217AAA308DBF9901A0FEB
:10175900788C7B191217AAA308DBF9901A2822C2E0
:10176900AF1217ED1217CA901A00740E1217AFA311
:1017790074091217AFA374151217AF901A03788062
:101789007B0A1217AEA308DBF9901A0F788C7B1924
:101799001217AEA308DBF91218001217DE901A28E7
:1017A90022E493F622E6438F01538FFDFFC3E583BD
:1017B900941C400122EF857CB7857DB7F0538FFEDD
:1017C90022438F02438F01857CB7857DB7901A0D1F
:1017D900F0538FFC22901A0D74A5F1AF901A0E7474
:1017E9005AF1AF227A3079D07820901A40F1AAE5DF
:1017F90020F709A3DAF7227A3079D0901A40E71254
:1018090017AF09A3DAF822AB74A875BB0102798076
:10181900BB02027981BB03027982BB04027994BBC2
:1018290005027983BB06027986BB07027992BB0858
:10183900027987BB0902799CBB0A027988BB0B0232
:101849007989E8F7227C051205BEDCFB22C2AF12BA
:1018590005CE1205D51205DC1205E31205AF1205F6
:0D186900CE1205D51205DC1205E31205AF05
:101876001205CE1205D51205DC1205E3D2AF22C23F
:10188600AF1205E31205DC1205D51205CE1205AF1F
:101896001205E31205DC1205D51205CE1205AF12AC
:1018A60005E31205DC1205D51205CED2AF22AE74C1
:1018B600AF75C2AF1205CE1205CE1205CE1205AF18
:1018C600DEF21205E31205AFDFF8D2AF2211561190
:1018D6004E114E75740175750175760011B47C054F
:1018E600AD5C1205BEC3ED955C70F5C3E55C940175
:1018F600400AC3E55C94FF40330219101110121719
:10190600681156C2AF75EF16114EDCD40576C3E5E5
:10191600769403500280C5114E0575E57414900047
:101926009F93F808C3E57598500280AD114E114E8D
:101936000574C3E574940C5002809B12105912175B
:0819460068C2AF75EF16114EE7
:0319FD000211D004
:101A00000E091507070104FFFF0A020101A55A018B
:101A100000B4FFFFFF03FF01FF25D078C804FF01DA
:091A200000FF0A010100FF00FFB4
:101A4000234F76736B794D5232304150726F2320A1
:101A500023424C48454C492346333930232020202B
:101A60002020202020202020202020202020202076
:101C0000C2AFC2D353D9BF7581C043B20343FF8073
:101C1000752438752503B1DC7529A5752AF175E29F
:101C20004043F18053A47F75D4FFD2877DFA7803B7
:101C300079E67C10752200752300901DE97B0675FE
:101C400024987525013087028145208708D8FBD963
:101C5000F9DCF781B7308708D8FBD9F9DCF781B711
:101C6000B19CE493A3C39A6004DDC381B7DBDBB10D
:101C70008E6002812E7B08E493FAA3B16FDBF87AC1
:101C800030B16F752200752300B18EEAFCEBFDC305
:101C9000ED94FE400EB18E8A278B28ED30E0048A49
:101CA000828B83B18E7AC270D8C3ED94FE601950D6
:101CB000CEBD002BEC600F7520007521FF7529004B
:101CC000752A000200008100A827A9280809D80465
:101CD000D90281DCB192EA89AAF281CE0D81A3C337
:101CE000ED94035053EDA2E092007AC5C3E58294CF
:101CF00000E583941C508A200010438F02438F011B
:101D00008529B7852AB7F0300029A827A92808090E
:101D1000438F01538FFDD804D902A133C3E58394C7
:101D20001C4003A3A11689AAE28529B7852AB7F02A
:101D3000A3A116538FFC817F7AC1BD030CE493A34A
:101D4000FAB153DCF8B14B817F8181AA22AB23B178
:101D50006FEBFAEA6222752608C3E52313F523E543
:101D60002213F52250066323A0632201D526EAB18F
:101D7000DCB1DC75260AEAF4200102D287300102C8
:101D8000C287B1DCC3134002C201D526EB22B19257
:101D9000EAFB208702A192308702A197752608AE40
:101DA00024AF25C3EF13FFEE13FEB1E0B1DCC3EAAD
:101DB000133087024480FA30E703632201C3E5232E
:101DC00013F523E52213F52250066323A0632201B5
:101DD000D526D9E52265236523F52222AE24AF2539
:101DE0000E0FDEFEDFFCD20122424C48656C6934E6
:071DF000373164F390060196
:00000001FF
